:020000040000FA
:0600000052EF03F01200B4
:0600080004EF04F01200F9
:060018000CEF04F01200E1
:02002A000000D4
:04002C006C5002E032
:10003000000E01D0010E00090BE0040100513C0B41
:10004000E842E8420D0802E131EF00F043EF00F032
:100050006C5002E0000E01D0010E040901E022D82C
:100060001200D9CFE6FFE1CFD9FFE6520001746B51
:10007000756B7A6B7B6BF9EC01F098D8E552E55221
:10008000E7CFD9FF1200020E0001745D09E164D8C8
:10009000040100BD02D0C80E01D0880E006F12000E
:1000A0001BEF01F0040E00017C5D09E112C46EFF3C
:1000B0006E50000802E2050E01D0030E7C6F0001B5
:1000C000740509E10AD8040104BD02D0C80E01D0AC
:1000D000880E046F12001BEF01F0D9CFE6FFE1CFCD
:1000E000D9FFE6520001080E7A5D000E7B5903E24B
:1000F0007AC0DFFF02D0080EDF6EDFCF05F4DF50DD
:10010000016AE8507A5F01507B5B180E786F040E2D
:10011000796FDF501CE000017DA307D076C0F6FFA9
:1001200077C0F7FF0800F55005D076C0E9FF77C02B
:10013000EAFFEF5078C0E9FF79C0EAFFEF6E0001F7
:10014000762B000E7723782B7923DF06E2D7E55252
:10015000E552E7CFD9FF1200D9CFE6FFE1CFD9FFB3
:10016000E65201C4DFFFDF5000017A257A6F000EEE
:100170007B217B6F180E766F040E776FDF5011E0D6
:1001800076C0E9FF77C0EAFFEF5078C0E9FF79C099
:10019000EAFFEF6E782B000E7923762B7723DF06AC
:1001A000EDD7E552E552E7CFD9FF120000017551B6
:1001B0000BE10401080E016F100E026F040E036FB5
:1001C000840E006F040123D0040110AF22D000017F
:1001D0007A510401165D00017B510401175904E2B4
:1001E00016C47AF017C47BF078DF0001010E746F3B
:1001F0000401080E016F100E026F040E036F800ED3
:10020000006F0401180E066F040E076FC80E046F0E
:1002100010D00001020E746F0401056BC80E046F4C
:100220000401080E016F180E026F040E036FC80E52
:10023000006F6D9812000001746B0401080E016FCD
:10024000100E026F040E036F880E006F0401046B22
:0202500012009A
:0E02520000016C6B1E0E716E706B716B0401FF
:10026000400E096F200E0A6F040E0B6F880E086F88
:100270000401200E0E6F040E0F6F400E0C6F120063
:10028000550EA76EAA0EA76EA682120067EC03F0A9
:100290000E0EE66EE66A1EEC03F0E552E55204012E
:1002A000226F0F0EE66EE66A1EEC03F0E552E55291
:1002B0000401236F5B0E246F120E256F120022C4FF
:1002C0006DF023C46EF024C46FF025C470F026C412
:1002D00071F01200940EA66E6DC0F6FF6EC0F7FFAF
:1002E0006FC0F8FFCDDFF86A840EA66E00016A6B5E
:1002F000400E6A5D24E26A51EA6A200FE96E040E3C
:10030000EA22EFCF03F06AC000F0016A026A6D5181
:100310000024F36E6E510120F46E6F510220F86ECE
:10032000F4CFF7FFF3CFF6FF03C0F5FF0C001F0E6D
:100330006A151F0801E1A4DF00016A2BD9D712005A
:10034000060E00017C5D54E36D50020B01E01200CB
:1003500000016C050DE104010CBF4AD00401400E00
:10036000096F0817087D880E081300016C6B1200D6
:10037000040108BF3DD000016A6B705171111DE08E
:10038000A9DF00017007000E715B0401020E206FEF
:10039000070E216F6DC022F46EC023F46FC024F4E9
:1003A00070C025F471C026F4400E00016D27000EC8
:1003B0006E236F23070E6A6F0ED004012051020ACC
:1003C00006E0020A08E162DF0001060E03D077DFD3
:1003D0000001010E6A6F0001010E6C6F6A5108E0A6
:1003E0006AC00DF4400E04010C170C7D880E0C132E
:0203F0001200F9
:0E03F20004011051600BE842E842E842E84284
:10040000E842000901E012001151080A39E0010A2E
:1004100035E00F0A0AE0030A01E012000001010EB4
:10042000756F0001040E7C6F12000001010E756FE4
:100430000401130507E10001060E766F060E776FC3
:10044000120E13D0020E135D07E10001180E766F35
:10045000060E776F200E09D0030E135D0AE100012E
:10046000380E766F060E776F040E00017A6F7B6B85
:1004700002D00001756B00017D8312004EEF02F087
:100480000001010E756F00017E0E766F000E776F12
:1004900000017D930001010E7A6F12000001010E30
:1004A000756F12C47EF00401125104E10001050EC3
:0E04B0007C6F12000001060E7C6F29EF01F038
:0204BE00080E26
:1004C0006D6E6DBAFED7686A110E696E0001020E7C
:1004D0007C6F12006850040B06E06950040B03E0C7
:1004E0006D92699468946850010B04E06950010BA7
:1004F00001E027D86850100B09E06950100B06E0A6
:10050000698468986D82A08A0300A19A6850200BC4
:1005100009E06950200B06E070A003D01BEC01F04D
:100520007090689A030E00017C5D01E209D068506A
:10053000080B06E06950080B03E016EC00F0689623
:100540001200686A7B0E696E6E6A160E706E68A67F
:1005500002D06896FCD76D981BEC01F000017E6B11
:080560000001030E7C6F120084
:080568002A0EF66E000EF76E7C
:10057000000EF86E00010900F550656F0900F55096
:10058000666F03E1656701D03DD00900F550606FEB
:100590000900F550616F0900F550626F090009000C
:1005A000F550E96E0900F550EA6E090009000900EE
:1005B000F550636F0900F550646F09000900F6CF2C
:1005C00067F0F7CF68F0F8CF69F060C0F6FF61C060
:1005D000F7FF62C0F8FF0001635302E1645307E0D4
:1005E0000900F550EE6E6307F8E26407F9D767C0BB
:1005F000F6FF68C0F7FF69C0F8FF00016507000E4D
:06060000665BBFD712008B
:0A0606001201000200000008D804F1
:100610000B00000000000001090220000101008021
:10062000320904000002000000000705010240003A
:0C063000000705810240000004030904DB
:04063C00D9CFE6FF2D
:10064000DACFE6FFE1CFD9FFE2CFDAFFFF0EE76EA8
:10065000FC0EDBCF00F0E75000160050A96EA69C00
:10066000A69EA680A850E552E5CFDAFFE7CFD9FFD6
:02067000120076
:0E067200A968A69CA69EA680120EA85C02E1B6
:1006800000EF04F0120EA86EA68440EC01F001D831
:100690001200140E6F6E5FEC02F06AEC02F0A0EC38
:0406A00001F0FBD793
:0C06A40013EE00F023EE00F0F86A059C55
:1006B000B4EC02F06AEC03F039EC03F0FBD7120063
:0E06C00000EE00F00F0EEE6AEA62FDD71200A7
:0206CE00A6B2D2
:0406D000FED712003F
:0206D400120012
:080800009490949249EF03F07B
:020000040030CA
:0100000020DF
:0100010002FC
:010002003EBF
:010003001EDE
:010005008179
:010006008178
:010008000FE8
:01000900C036
:01000A000FE6
:01000B00E014
:01000C000FE4
:01000D0040B2
:00000001FF
